:100000000C9436030C945E030C945E030C945E0314
:100010000C945E030C945E030C945E030C945E03DC
:100020000C945E030C945E030C94792C0C941C2BA2
:100030000C945E030C945E030C945E030C945E03BC
:100040000C945E030C945E030C945E030C945E03AC
:100050000C94A00A0C945E030C945E030C9474033D
:100060000C945E030C945E030C945E030C945E038C
:100070000C945E030C945E030C945E030C945E037C
:100080000C945E030C945E030C945E030C945E036C
:100090000C945E030C945E030C945E030C945E035C
:1000A0000C945E030C945E030C945E032E004C00D3
:1000B0002A00E10047C900001E00140004001D00D2
:1000C00034004D001F001A0016001B00E1022A0038
:1000D000200008000700060050002C002100150039
:1000E000090019004F004A00220017000A0005000D
:1000F000000076C2500001440000E30B0000E30062
:100100004F0001440000E2090000E20023001C004F
:100110000B00110000003AC0240018000D00100070
:1001200052004B0025000C000E0036005100280044
:10013000260012000F0037002F002B0027001300AD
:1001400045CA380030004E002D00310045C3E5009F
:100150002B4400002900000000000000FFFF000009
:100160003A001E0820082208000000003B001F087B
:1001700021082308000000003C002F0826082F005B
:10018000000000003D00300827083000000000009B
:100190003E00310835003508000000000000FFFF78
:1001A00000000000000000000000FFFF0000000051
:1001B000000000003F005200510024080000000031
:1001C0004000240021001E00000000004100250026
:1001D00022001F00370000004200260023002000FC
:1001E0002700000043002508000031002E00000019
:1001F0004400450000000000FFFF00000000000078
:1002000000000000000000000000000000000000EE
:10021000000000000000000004500000000000008A
:10022000000001500250000041500000000000009A
:1002300008500000425000000000000000000000D4
:1002400000000000000000000000000000000000AE
:10025000000000000000000000000000000000009E
:10026000000000000000000000000000000000008E
:10027000E9480000000000000000B648EA4800001D
:10028000000000000000B548E24800000000000047
:10029000FFFF00000000000000000000CD4800004B
:1002A00000000000302E31312E302B3237007665C1
:1002B0007273696F6E0076657273696F6E00050107
:1002C0000906A101050719E029E7150025017501B7
:1002D000950881029501750881019505750105084C
:1002E000190129059102950175039101950675087B
:1002F000150025FF0507190029FF8100C0050C091D
:1003000001A1018504150026FF0319002AFF0395AA
:100310000475108100C005010906A10185080507C3
:1003200019E029E7150025017501950881020508E6
:1003300019012908950875019102050775049501B1
:100340008101190429DD15002501750195D9810266
:10035000750395018101C005010980A1018505157D
:100360000026FF00190029FF950175088100C0745F
:10037000726967676572006D6170006D6163726FAD
:10038000732E006D6163726F732E6D61700A6D6103
:1003900063726F732E747269676765720044796E59
:1003A000616D69634D6163726F7300657363617042
:1003B000655F6F6E6573686F742E63616E63656CE5
:1003C0005F6B6579006573636170655F6F6E657300
:1003D000686F742E63616E63656C5F6B6579004551
:1003E00073636170654F6E6553686F740065657007
:1003F000726F6D2E657261736500656570726F6DE9
:100400002E6672656500656570726F6D2E636F6E26
:1004100074656E747300656570726F6D2E636F6EB8
:1004200074656E74730A656570726F6D2E667265A1
:10043000650A656570726F6D2E6572617365002F58
:10044000006372630076657273696F6E0076616C2B
:1004500069643F0064656661756C744C61796572AE
:100460000073657474696E67732E007365747469C4
:100470006E67732E64656661756C744C6179657224
:100480000A73657474696E67732E76616C69643F74
:100490000A73657474696E67732E76657273696F1B
:1004A0006E0A73657474696E67732E63726300639A
:1004B0007573746F6D0064656661756C74006F6E42
:1004C0006C79437573746F6D006B65796D61702E17
:1004D000006B65796D61702E637573746F6D0A6B57
:1004E00065796D61702E64656661756C740A6B6503
:1004F000796D61702E6F6E6C79437573746F6D00DA
:10050000454550524F4D4B65796D61700066616C89
:100510007365007472756500706C7567696E730041
:100520006465766963652E72657365740068656CD1
:10053000700A6465766963652E72657365740A7006
:100540006C7567696E730068656C70000D0A2E002B
:100550004D6F7573654B657973004F6E6553686FAA
:10056000740051756B657973005370616365436105
:1005700064657400080B0002020200000904000018
:1005800001020200000524001001052401010104FC
:100590002402060524060001070581031000400916
:1005A000040100020A0000000705020240000007E3
:1005B00005830240000012010002EF020140EDFE3F
:1005C00007130001010203014572676F446F782031
:1005D000455A004572676F446F7820455A000403FE
:1005E000090405010902A10185010509190129086C
:1005F00015002501950875018102050109300931B1
:1006000009381581257F750895038106050C0A3880
:10061000021581257F750895018106C00501090233
:10062000A101050919012908150025019508750181
:10063000810205010930093116000026FF7F75107F
:100640009502810209381581257F7508950181067B
:10065000C000320A3E0FD70FCB102A11ED16121A26
:100660006F2379258726212DFC2ED02F11241FBE24
:10067000CFEFDAE0DEBFCDBF11E0A0E0B1E0EEE603
:10068000F1E602C005900D92AC3AB107D9F725E02A
:10069000ACEAB1E001C01D92A13BB207E1F713E063
:1006A000C6E3D3E004C02197FE010E941F30C93287
:1006B000D107C9F70E9461030C94B5300C94000077
:1006C00008950E9433040E94600389EB94E00E9425
:1006D000F12C0E94C205C0E0D0E00E94DB0520970B
:1006E000E1F30E940000F9CF1F920F920FB60F9214
:1006F00011242F933F938F939F93AF93BF93809138
:10070000AD019091AE01A091AF01B091B0013091D7
:10071000AC0123E0230F2D3758F50196A11DB11D23
:100720002093AC018093AD019093AE01A093AF01F3
:10073000B093B0018091B1019091B201A091B30149
:10074000B091B4010196A11DB11D8093B1019093A8
:10075000B201A093B301B093B401BF91AF919F9147
:100760008F913F912F910F900FBE0F901F90189572
:1007700026E8230F0296A11DB11DD2CF2FB7F89402
:100780006091AD017091AE018091AF019091B00187
:100790002FBF08953FB7F8948091B1019091B201B5
:1007A000A091B301B091B40126B5A89B05C02F3F1D
:1007B00019F00196A11DB11D3FBFBA2FA92F982F87
:1007C0008827BC01CD01620F711D811D911D42E082
:1007D000660F771F881F991F4A95D1F708958F924A
:1007E0009F92AF92BF92CF92DF92EF92FF926B01F6
:1007F0007C010E94CA034B015C01C114D104E104D5
:10080000F104E9F00E94202D0E94CA0368197909B9
:100810008A099B09683E73408105910570F321E0C8
:10082000C21AD108E108F10888EE880E83E0981E0C
:10083000A11CB11CC114D104E104F10429F7FF90FB
:10084000EF90DF90CF90BF90AF909F908F900895E2
:100850008230910538F0880F991F880F991F0597EE
:100860000197F1F70895789484B5826084BD84B5CA
:10087000816084BD85B5826085BD85B5816085BD9B
:10088000EEE6F0E0808181608083E1E8F0E01082B4
:10089000808182608083808181608083E0E8F0E0F5
:1008A000808181608083E1E9F0E0808182608083E3
:1008B000808181608083E0E9F0E0808181608083D5
:1008C000E1ECF0E0808184608083808182608083BD
:1008D000808181608083E3ECF0E0808181608083AF
:1008E000E0ECF0E0808182608083E2ECF0E08081E7
:1008F00081608083EAE7F0E080818460808380818A
:100900008260808380818160808380818068808331
:10091000089508958AE0E7E5F1E0DB0101900D928A
:100920008A95E1F78AE008958AEB93E00E948718A0
:1009300085EF93E00E9430208BE294E00E94E42354
:1009400083E191E00E94BD1E8CEA93E00E94F414C2
:1009500087E593E00E94D61280EE93E00E94821A0F
:1009600080E0089580EB93E00E94E8158AEB93E025
:100970000E947D188CEA93E00E94B41480EE93E00C
:100980000E94971A80E0089580EB93E00E94E5169C
:1009900080E00895CF93DF93EC01BC0185EF93E0F5
:1009A0000E94C022811107C0BE018BE294E0DF915A
:1009B000CF910C940125DF91CF910895CF93DF93D0
:1009C000EC01BC0183E191E00E94731F811115C00D
:1009D000BE0186E091E00E945D1581110EC0BE014E
:1009E00087E593E00E94B312811107C0BE0180EE3B
:1009F00093E0DF91CF910C940D1BDF91CF9108957F
:100A0000BC0180EE93E00C94C71A0F931F93CF9311
:100A10008C01BC018AEB93E00E942919C82F811137
:100A20004BC0B8018FEB93E00E94E519C82F8111EC
:100A300043C0B8018EEA93E00E940317C82F8111CA
:100A40003BC0B8018FEA93E00E948517C82F81113F
:100A500033C0B8018CEA93E00E940915C82F8111B8
:100A60002BC0B80187E593E00E940413C82F8111C1
:100A700023C046EB52E0B8018FEB93E00E94D019FF
:100A800081111AC06EEA72E0C8010E946030892BA1
:100A900099F464EA72E08CE594E00E94872784E68A
:100AA00090E00E94280460E28CE594E00E94AB276D
:100AB00084E690E00E9428048C2FCF911F910F9123
:100AC000089580E00895BC018CE993E00C947114C2
:100AD000CF93DF93EC01BC0183E191E00E94611FA1
:100AE000BE0180EE93E00E94C91B80E0DF91CF91B0
:100AF00008958FEB93E00E94151A85EF93E00E9412
:100B000031238BE294E00E949F2483E191E00E94D4
:100B1000D21E80EE93E00E94811B80E00895CF9367
:100B2000C0E040E06C2F8EE292E00E942F0CCF5F7D
:100B3000C430B9F7C1E041E06C2F8EE292E00E9430
:100B40002F0C2FEF80E792E0215080409040E1F79A
:100B500000C00000CF5FC43071F7C1E040E06C2FEF
:100B60008EE292E00E942F0C2FEF80E792E021505E
:100B700080409040E1F700C00000CF5FC43071F7C3
:100B8000CF91089580916201909163010E949D062A
:100B900085E00E94A71881E080932B0460E071E05B
:100BA00087E593E00E94EB120E948F058091B403C9
:100BB0008F770C94420980916201909163010C94AB
:100BC000BB0681EC92E00E94820E811104C081EC90
:100BD00092E00C94200F80E093E00E94BB1082EE24
:100BE00092E00C949C0F81EC92E00E94820E8111A5
:100BF00004C081EC92E00C94850E80E093E00E94AA
:100C0000071082EE92E00C94AF0FCF93C82F81ECC7
:100C100092E00E94820E6C2F811105C081EC92E05F
:100C2000CF910C94C10E80E093E0CF910C946B10A7
:100C3000CF93C82F83FF03C081EE0E940506C0FF3B
:100C400003C080EE0E940506C1FF03C082EE0E9431
:100C50000506C2FF03C086EE0E940506C4FF04C05D
:100C600083EECF910C940506CF910895CF93C82FB2
:100C7000892F0E9418068C2FCF910C940506CF93D4
:100C8000C82F81EC92E00E94820E6C2F811105C06A
:100C900081EC92E0CF910C94E80E80E093E0CF914C
:100CA0000C949210FC019081DB018C91981305C08B
:100CB00081E0218111969C91291380E008951F9372
:100CC000CF93DF9300D000D0CDB7DEB7182F843597
:100CD00068F5E82FF0E0EE0FFF1FEC53FB4F80812B
:100CE00091819C838B838FEF89838A83BE016F5FA1
:100CF0007F4FCE0103960E945206882369F0A12FF0
:100D0000B0E0A554BE4FE0910201F0910301612FC4
:100D10008C9109958B839C838B819C810F900F9084
:100D20000F900F90DF91CF911F91089510926C0555
:100D300010926D05ECE6F5E0D2CF8EE292E00E94D3
:100D40004A0A40E855E260E070E08CE594E00E94D9
:100D500081260E9489040E94B204E4ECF4E085E557
:100D60009FEF815021F0908391833296FACF8AEBE6
:100D700091E00C9440090E94BE036093B601709309
:100D8000B7018093B8019093B9010E94C4048EE228
:100D900092E00E941E0C0C9479051F93CF93DF9371
:100DA000C62F172F862F972F0E940005823009F13A
:100DB000812F807C61F480E28C0F883008F010E095
:100DC0008C2F912FDF91CF911F910C943606812F9C
:100DD000887C883471F4612F70E0762F66276C0F61
:100DE000711D737082EE92E0DF91CF911F910C9490
:100DF000870FDF91CF911F9108958F929F92BF929D
:100E0000CF92DF92EF92FF920F931F93CF93DF93D6
:100E100000D000D000D0CDB7DEB77C016B010E94BE
:100E2000E10510E000E0BB24BA940435110599F106
:100E3000F6019081901729F1043530F5F801EE0F95
:100E4000FF1FEC53FB4F808091809E828D82BB827E
:100E5000BC82BE016D5F7F4FCE0105960E94520697
:100E600081110FC019821A82BE016F5F7F4FCE01C0
:100E700005960E945206811104C0B401C7010E9468
:100E8000CD060F5F1F4FD1CF10926C0510926D05EC
:100E9000ECE6F5E0D8CF26960FB6F894DEBF0FBE8D
:100EA000CDBFDF91CF911F910F91FF90EF90DF9019
:100EB000CF90BF909F908F900895EF92FF920F93E5
:100EC0001F93CF93DF938C01EB01898181FF43C096
:100ED00080FD41C08B81807CF1F588818093010188
:100EE000FA8081EC92E00E94820E6F2D81112EC05B
:100EF00081EC92E00E94310F882301F1FB80EA80AF
:100F0000F3FE03C081EE0E943F06F0FE03C080EEB8
:100F10000E943F06F1FE03C082EE0E943F06F2FEF1
:100F200003C086EE0E943F06F4FE03C083EE0E94DB
:100F30003F068E2D0E943F060E94F3058B81882379
:100F400079F00E9418060E94F3050AC080E093E041
:100F50000E945510D1CFE09101018881E81317C09C
:100F6000898181FF07C080FD05C06A817B81C8013E
:100F70000E94CD06CE010E9463058230E9F0DF9128
:100F8000CF911F910F91FF90EF900C94F305E435F2
:100F900060F4F0E0EE0FFF1FEC53FB4F8181982FC0
:100FA000907CF1F60E941806DBCF10926C0510922F
:100FB0006D05ECE6F5E0F2CFDF91CF911F910F9137
:100FC000FF90EF900895FF920F931F93CF93DF93BD
:100FD000CDB7DEB72D970FB6F894DEBF0FBECDBFED
:100FE0008C0129873A874B875C876D87243548F4C5
:100FF00030FF61C031FD5FC089850E945F069C871C
:101000008B87CE0109960E94DE04823009F447C026
:10101000E985E43568F49A85F0E0EE0FFF1FEC53A4
:10102000FB4F90FF55C091FD53C09FEF908391837C
:10103000811135C01F821886BE01695F7F4FCE01C6
:101040000B960E94520681112AC01D821E82BE018B
:101050006B5F7F4FCE010B960E94520681111FC01D
:10106000FF24FA94FB82FC82BE016D5F7F4FCE01AC
:101070000B960E945206811112C0F982FA82BE01BB
:101080006F5F7F4FCE010B960E945206811107C001
:101090008C85843409F5CE0109960E94D3092D96DA
:1010A0000FB6F894DEBF0FBECDBFDF91CF911F9179
:1010B0000F91FF9008958FEF89838A83BE016F5F40
:1010C0007F4FCE010B960E945206811195CF99CF8A
:1010D0009C852B852083ABCF8F7C8134B9F48A85A6
:1010E0001B8581FF0AC080FD08C0612F88E493E062
:1010F0000E94121110933302D2CF809133028113D8
:10110000CECF88E493E00E941011C9CFBE01675F83
:101110007F4FC8010E94FD06BE01675F7F4FC80177
:101120000E945D07CE0109960E946805B8CFEF9234
:10113000FF920F931F93CF93DF9300D000D000D086
:101140001F92CDB7DEB7022F2B833C834D835E8386
:101150006F83243508F042C07C01832F817031FFFA
:1011600022C081113BC08FEF89838A83BE016F5FEC
:101170007F4FCE0105960E945206882329F0802FCA
:101180000E945F069E838D83CE0103960E94CA044F
:10119000811124C02B813C814D815E816F81C7010B
:1011A0000E94E3071BC08823C9F010E0000F111F45
:1011B0000C531B4FF801808191819E838D8319828E
:1011C0001A82BE016F5F7F4FCE0105960E945206C4
:1011D0008823D1F28FEFF8018083818327960FB6A1
:1011E000F894DEBF0FBECDBFDF91CF911F910F915D
:1011F000FF90EF90089570E094E5899F600D711D58
:101200001124660F771FFB01E455FF4F8491FB010A
:10121000E355FF4F94910895EF92FF920F931F9320
:10122000CF93DF93EBEBF1E084E5DF011D928A952C
:10123000E9F77F0110E01435E1F0C0910401D0E03E
:10124000C15FDD4FB2E0CF30DB0771F00A91E09172
:101250000201F0910301612F802F09958F3F11F456
:101260009F3F81F3F70100831F5FFFEFEF1AFF0A33
:10127000E2CFDF91CF911F910F91FF90EF900895F2
:101280000C940C0990910001891708F080E091E01E
:101290009093040180930F020E940C090C94610545
:1012A0004091040150E090E0682F70E0292F092E52
:1012B000000C330B2417350764F4215F3D4FF9010F
:1012C0002081022E000C330B2617370721F09F5F79
:1012D000EDCF80E0089581E00895CF9390910001D3
:1012E0008917A0F4C82F0E94500981110FC0E09106
:1012F000040181E08E0F80930401F0E0E15FFD4F77
:10130000C0830E940C09CF910C946105CF91089580
:10131000CF93DF93D82F0E945009882381F1C09189
:101320000401C23028F480E0DF91CF910C9442098F
:10133000EFE0F2E090E080E02D2F30E04191042ECC
:10134000000C550BBC016F5F7F4F4217530799F498
:101350004C2F50E0481B590B615F7D4F815F9D4FC3
:101360000E948D30C150C09304010E940C09DF918E
:10137000CF910C946105CB016C1700F3F6CFDF9190
:10138000CF910895E0910401F0E0E25FFD4F80818C
:101390008F5F0C946D09E0910401F0E0E25FFD4F76
:1013A00080810C948809CF93DF93FC01C2819181E5
:1013B000292F2270C43558F0222309F450C090FD23
:1013C0004EC08CEA8C0FDF91CF910C944209CA3247
:1013D000C8F1D6EDDC0FD13251F0D23281F42223A4
:1013E00051F090FD08C0DF91CF910C94C2092223E7
:1013F000D1F390FDF8CFDF91CF910C94CB0921115F
:1014000010C0A4ECB4E085E58150B9F09C91C913FB
:1014100006C011962C9111979381291701F112960C
:10142000F3CF90FDEECF8D2F0E945009811117C090
:101430008D2FDF91CF910C946D098D2FDF91CF917E
:101440000C948809222359F090FD09C08C2F0E942A
:101450005009882311F08C2FF1CF8C2FEACFDF9128
:10146000CF910895EEE2F2E0158285E0858780E273
:101470008687089581EC92E00E94270F80E093E038
:101480000E94C11082EE92E00E94D50F88E493E0A2
:101490000C940E11EF92FF920F931F93CF93DF9353
:1014A0007C010FB6F894A8958091600088618093C4
:1014B0006000109260000FBE64E670E080E090E093
:1014C0000E94EF0300E810E089EAF8018083C1E898
:1014D000D0E089E0888324982C983F988AB18F7C4B
:1014E0008AB96E98479A8BB180638BB9769AC70197
:1014F0000E960E94840C8FE090E090938900809378
:10150000880090938B0080938A0090938D00809345
:101510008C0080E18883F801108280E295E390934B
:1015200087008093860081E1888381E080936F004B
:10153000DF91CF911F910F91FF90EF900C943A0A99
:101540001F920F920FB60F9211248F9381E0809318
:1015500005018F910F900FBE0F901F9018958F92DD
:101560009F92AF92BF92CF92DF92EF92FF920F9332
:101570001F93CF93DF936C01109205015C018EE005
:10158000A80EB11CC5010E94240DE601AB964601D0
:10159000EDE18E0E911CF12CE12CABC081508883C3
:1015A00012E002E020E090E08981882321F0815060
:1015B0008983122F092F8A818111C2C01460012FE3
:1015C0008B818111C3C01860012F8C818111B5C03E
:1015D0001061012F8D818111ADC01062012FB70103
:1015E000C5010E94E40CF401908110951923802319
:1015F000812B982790FF03C0F6012585288391FF52
:1016000003C0F6012585298392FF03C0F6012585D5
:101610002A8393FF03C0F60125852B8394FF03C023
:10162000F60125852C8395FF03C0F60195859D83E2
:10163000F40181934F01B701695F7F4F8AA5882329
:1016400009F473C081508AA712E002E020E090E024
:101650008BA5882321F081508BA7122F092F8CA5F1
:10166000811160C01460012F8DA5811158C01860D0
:10167000012F8EA5811150C01061012F8FA58111FE
:1016800048C01062012FC5010E94E40CF40196814C
:10169000109519238023812B982790FF03C0F60112
:1016A00025852AA791FF03C0F60125852BA792FF68
:1016B00003C0F60125852CA793FF03C0F6012585FD
:1016C0002DA794FF03C0F60125852EA795FF03C023
:1016D000F60195859FA7F4018683B701C5010E9495
:1016E000CA0CFFEFEF1AFF0A269687E0E816F1040E
:1016F00081F1B701C5010E94A10CB701C5010E948B
:10170000CA0C888181114ACF13E003E021E091E007
:101710004BCF81508FA7B7CF81508EA7AFCF8150CD
:101720008DA7A7CF81508CA79FCF13E003E021E0C6
:1017300091E08ECF81508D8352CF81508C834ACFE0
:1017400081508A838B81882309F43DCF81508B831C
:101750003CCFDF91CF911F910F91FF90EF90DF90E1
:10176000CF90BF90AF909F908F900895CF92DF92CF
:10177000EF92FF920F931F93CF93DF9300D000D08F
:101780001F92CDB7DEB70F967C01D12CCC24CA9422
:1017900010E000E0F70126851BC03230A1F4609113
:1017A000C3046F5F6093C3042D2D200F29833A83F8
:1017B000CB82CC826D834FEF5FEF85EB91E00E948F
:1017C0009708F70126850F5F1F4F0630110501F1BD
:1017D000F701808190E0002E02C0959587950A94CC
:1017E000E2F7382F3170822F90E0002E02C09595DD
:1017F00087950A94E2F7880F991F8270382B811120
:10180000CCCF30FDCCCF0F5F1F4F0630110501F755
:10181000F70121937F01F6E0DF0E84E5D812B8CFFF
:101820000F900F900F900F900F90DF91CF911F911D
:101830000F91FF90EF90DF90CF900895CF93DF93BB
:10184000EC0180910501882329F010920501CE0159
:101850000E94AF0ACE01DF91CF910C94B60B6C5F62
:1018600081E090E001C0880F6A95EAF794B14423C3
:1018700031F0982B94B995B1892B85B9089580954D
:10188000982394B995B1892385B90895CF930E947F
:10189000630D68EE73E080E090E00E94EF0380E467
:1018A0000E94690DC82F81112AC080E00E94930D0B
:1018B000C82F811124C080E00E94930DC82F811190
:1018C0001EC08FE30E94930DC82F811118C00E9483
:1018D0008B0D80E40E94690DC82F811110C08CE02F
:1018E0000E94930DC82F81110AC080E00E94930DC1
:1018F000C82F811104C08FE30E94930DC82F0E944E
:101900008B0D8C2FCF910895CF93DF93EC010E9424
:10191000460C888380B38C7080BB81B3836F81BB9E
:1019200084B18F6084B985B18F6085B98AB18C60CC
:101930008AB98BB18C608BB93E9A469ADF91CF9170
:1019400008951F93CF93DF93FC012081222321F080
:10195000DF91CF911F910895162FEC0180E40E9432
:10196000690D8883882329F0DF91CF911F910C9412
:101970008B0D82E10E94930D88838111F5CF81E068
:1019800090E001C0880F1A95EAF780950E94930DA8
:101990008883EACFFB01EC59FE4F8081E82FF0E00D
:1019A000F595E795F595E795F595E795F595E7951F
:1019B00092A18F7021E030E001C0220F8A95EAF7F2
:1019C000892F822782A308950F931F93CF936730A7
:1019D000710554F4FC01C081CC23A1F0C0E08C2F30
:1019E000CF911F910F9108958FB1CFB1C695C69534
:1019F000CC738370C82BC095CF738C2FCF911F9160
:101A00000F9108958C0180E40E94690DF801808394
:101A1000882339F00E948B0D8C2FCF911F910F914D
:101A2000089583E10E94930DF80180838111F2CF24
:101A300081E40E94690DF80180838111EBCF0E943F
:101A4000A40DC82FC095E6CF0F931F93CF93DF93BC
:101A5000EC018091AD0281110DC00E94BE03609324
:101A6000B5027093B6028093B7029093B80281E0FA
:101A70008093AD028881882309F10E94BE03009102
:101A8000B5021091B6022091B7023091B802601BE6
:101A9000710B820B930B683873418105910570F0CF
:101AA000CE010E94460C88830E94BE036093B5025B
:101AB0007093B6028093B7029093B802DF91CF91F2
:101AC0001F910F9108951092B9008AE08093B80099
:101AD000089594EA9093BC009091BC0097FFFCCFCE
:101AE0009091B900987F983021F0903111F081E009
:101AF00008958093BB0084E88093BC008091BC0073
:101B000087FFFCCF8091B900887F883111F0803445
:101B100071F780E0089584E98093BC008091BC0057
:101B200084FDFCCF08958093BB0084E88093BC00C3
:101B30008091BC0087FFFCCF9091B900987F81E035
:101B4000983209F480E0089584E88093BC00809185
:101B5000BC0087FFFCCF8091BB000895FC0182810F
:101B60008F5BFB01808381E00895CF93DF93CDB736
:101B7000DEB769970FB6F894DEBF0FBECDBFFC018C
:101B8000DB019C919F5F9C939E012D5F3F4F81E104
:101B9000D9011D928A95E9F729E0298384E08A8397
:101BA00091E09D8383E08E839F8398872A8721E23B
:101BB0002B879C879D879F8722E2288B2FE3298B89
:101BC00027E02B8B25E02C8B8E8B20E430E0388FA8
:101BD0002F8B998F82818B83838180688D8B49E1E4
:101BE00050E0BE016F5F7F4F80E00E94CB2A699674
:101BF0000FB6F894DEBF0FBECDBFDF91CF91089531
:101C0000FC01DB018C918138A9F413968C91139718
:101C1000823281F4228114968D919C9128171906A5
:101C200049F48285848F4FE350E06EEB72E080E8E8
:101C30000C94CB2A90E080E00895FC01DB01228126
:101C400014968D919C9115972817190681F5119678
:101C50008C9111979C91913A69F4813029F08330ED
:101C600029F4848D8093F10081E008958230F9F4A5
:101C7000858DF8CF9132D9F48B3021F412968C9166
:101C8000848FF2CF8A3011F4158EEECF893079F43B
:101C9000CF0116962D913C91179713964C91423097
:101CA00041F461E070E04E962130310551F080E062
:101CB00008954130E1F728303105C9F768E070E058
:101CC0000B960E94F12AD0CFCF93DF93EC0181E0F5
:101CD0008C838D839E01255E3F4F3F832E83198623
:101CE00018862FE631E0398328836A876C8F8D8FC1
:101CF0001E8E81EC8B8F0E946427BE01DF91CF91F5
:101D00000C942027FC01848D0895EF92FF920F938D
:101D10001F93CF93DF938C01EC012B967C0183E121
:101D2000E80EF11C48E050E0BE01C7010E94773088
:101D3000892B21F1F801838148E050E0BE018064E5
:101D40000E941A2A8C01E091E002F091E1023097A2
:101D500031F09C0148E050E0BE0182E0099588E046
:101D6000FE01D70101900D928A95E1F7C801DF913C
:101D7000CF911F910F91FF90EF9008950FEF1FEFFC
:101D8000F5CFFC0180E2860F883070F4605E770B3F
:101D900021E030E001C0220F6A95EAF78385822BAB
:101DA000838781E090E00895DF011D9690E080E058
:101DB0002D912617B1F3211104C0E80FF91F658793
:101DC000F0CF01968630910599F790E080E0089574
:101DD000CF93DF9320E2260F283090F4605E770BDC
:101DE00021E030E001C0220F6A95EAF72095FC015E
:101DF00033852323238781E090E0DF91CF910895FD
:101E0000DC011D969C012D5E3F4FFD014191461363
:101E100003C0EF0121971882E217F307B9F720E01A
:101E20003D91332349F0EC01C20FD11D4D853D8713
:101E3000ED01219748832F5FAE17BF0789F7DBCFEE
:101E40000B9628E0FC0111922A95E9F70895CF93AB
:101E5000DF93EC010E94200FCE01DF91CF910C9413
:101E6000850EFC013D9643962191261729F0E8172F
:101E7000F907D1F780E0089581E008952091B90233
:101E80003091BA024091BB025091BC026091BD02F8
:101E90007091BE028091BF029091C002A1E00E94A9
:101EA0003F302093B9023093BA024093BB02509363
:101EB000BC026093BD027093BE028093BF029093F8
:101EC000C0020E944B3029F461E081EC92E00C9456
:101ED000640E08958091F202811113C01092FB02EA
:101EE0001092FA028DEF92E09093FD028093FC0233
:101EF00089E190E09093FF028093FE0281E080935D
:101F0000F2020E94882E6AEF72E00C94F52DFC011B
:101F100030E020E041915191452B41F4220F331FD5
:101F2000280F391FF9017183608308952F5F3F4F98
:101F30002430310579F7089528E0FC0111922A95A3
:101F4000E9F70895CF93DF93EC010E94882E28E0F3
:101F500030E0AE0164E0DF91CF910C94452E0F93F9
:101F60001F93CF93DF93EC018C01085F1F4F48E074
:101F700050E0BC01C8010E947730892B51F0CE019E
:101F80000E94A20F88E0FE01D80101900D928A956F
:101F9000E1F7DF91CF911F910F91089528E0FC01A7
:101FA00011922A95E9F70C94AF0F0C94CE0F82EEA4
:101FB00092E00C946A0F80913A03811113C0109241
:101FC00043031092420386E193E09093450380938C
:101FD000440381E490E0909347038093460381E0BB
:101FE00080933A030E94882E62E473E00C94F52DEE
:101FF000CF93DF93EC010E94882EAE01435E5F4FCA
:102000002DE130E068E0DF91CF910C94452EEF9206
:10201000FF920F931F93CF93DF93EC01F8808D8D88
:102020008E010F5F1F4F8F15D9F0F801AE01435E8F
:102030005F4F20E0858D30813196932F90959823C6
:1020400019F08323848F21E0E417F50799F7222301
:1020500019F0CE010E94F80FFD8ECE010E94F80FFC
:102060007E018EE1E80EF11C4CE150E0B801C701A1
:102070000E947730892B81F08CE1F801D701019023
:102080000D928A95E1F7CE01DF91CF911F910F91CB
:10209000FF90EF900C94F80F8FEF9FEFDF91CF91AF
:1020A0001F910F91FF90EF9008956E3D90F4E62FF1
:1020B000E695E695E695E80FF92FF11D677021E0AA
:1020C00030E001C0220F6A95EAF79181922381E006
:1020D00009F480E008956E3DA0F4E62FE695E695BC
:1020E000E695E80FF92FF11D677021E030E001C09F
:1020F000220F6A95EAF78181822B818381E090E04B
:102100000895605E683058F441E050E001C0440F2B
:102110006A95EAF7FC012081242B2083EFCF90E021
:1021200080E008956E3DA8F4E62FE695E695E695E5
:10213000E80FF92FF11D677021E030E001C0220F98
:102140006A95EAF7209581812823218381E090E038
:102150000895605E683060F421E030E001C0220F35
:102160006A95EAF72095FC01308123232083EECF86
:1021700090E080E008952DE1FC0111922A95E9F7A5
:102180000895CF93DF93EC010E94BB10CE01DF9145
:10219000CF910C94F80F80E093E00C94DB0F8091CA
:1021A0004903811113C0109252031092510387E525
:1021B00093E0909354038093530388E190E09093CD
:1021C00056038093550381E0809349030E94882E33
:1021D00061E573E00C94F52D0F931F93CF93DF937C
:1021E000EB018A010E94882E9801AE0165E0DF9123
:1021F000CF911F910F910C94452ECF93DF931F9297
:10220000CDB7DEB7198241E050E0BE016F5F7F4F6E
:102210000E94EC100F90DF91CF9108950C94FD1067
:102220000C94FD10CF93DF931F92CDB7DEB7698377
:10223000633841F489EB94E00E94042D0F90DF9104
:10224000CF91089541E050E0BE016F5F7F4F0E9443
:10225000EC10F4CF88E493E00C94CF100C949F30F2
:102260008F929F92AF92BF92CF92DF92EF92FF92A6
:102270000F931F93CF93DF938C01FC01E080F180DB
:1022800015821482C280D380CE0CDF1C4701B12C92
:102290008C149D0408F04BC0E4012196C4010E94F7
:1022A0002E118E3008F043C0E82FF0E0E65AFE4EC3
:1022B0000C941F308911681168116C116C116C112C
:1022C0006811681168116A116A116A116F117E1123
:1022D000E40122964E01DCCFE4012396FBCF4E01B0
:1022E000CE010E942E11A82E2296C40101960E94B2
:1022F0002E11A110F4CF8111F2CFECCF2C2F9D2FF6
:102300002196822F0E942E112C2F9D2F8111F8CF04
:10231000E1CFB394EB2DF0E03296EE0FFF1FE00F0C
:10232000F11FCE018E199F0991838083D3CF8B2D0E
:10233000DF91CF911F910F91FF90EF90DF90CF90A1
:10234000BF90AF909F908F9008958F929F92AF9281
:10235000BF92CF92DF92EF92FF920F931F93CF9392
:10236000DF93FC01EC5BFF4F2081621708F0DFC0B8
:102370007C01E62FF0E03296EE0FFF1FEE0DFF1D01
:10238000D7010D911C9180819181080F191FD12CCB
:10239000F7018081918122813381820F931F081779
:1023A000190708F0C4C0E8012196C8010E942E1147
:1023B00081508D3008F0BBC0E82FF0E0EE51FE4EAA
:1023C0000C941F300E121D1229123A124B125C127D
:1023D00068127412151215121512EF1180128D2C3D
:1023E000912CB12CA12CCE010E942E11C82E8E0151
:1023F0000E5F1F4FCE0101960E942E11811102C067
:10240000CC2091F0682F7C2D8CE993E00E944C1435
:10241000C501B4010E94EF03E801E5CF0E5F1F4F35
:10242000CE010E942E11D82EE8016D2D70E090E0B3
:1024300080E00E94EF038E01ABCF0E5F1F4FCE01F5
:102440000E942E11682F70E090E080E00E94EF0360
:10245000EBCFCE010E942E11C82EE8012396C801B1
:1024600002960E942E11682F7C2D8CE993E00E9429
:10247000A813DBCFCE010E942E11C82EE8012396AF
:10248000C80102960E942E11682F7C2D8CE993E0E2
:102490000E94E313CACFCE010E942E11C82EE8017C
:1024A0002396C80102960E942E11682F7C2D8CE97C
:1024B00093E00E944C14B9CF0E5F1F4FCE010E94D3
:1024C0002E11682F70E08CE993E00E94A813ACCF26
:1024D0000E5F1F4FCE010E942E11682F70E08CE915
:1024E00093E00E94E313A0CF0E5F1F4FCE010E9426
:1024F0002E11682F70E08CE993E00E944C1494CF69
:10250000CE018D2C912CB12CA12C21960E942E1144
:10251000882309F48ACF682F70E08CE993E00E9449
:102520004C14C501B4010E94EF03CE01EECFDF9140
:10253000CF911F910F91FF90EF90DF90CF90BF90C0
:10254000AF909F908F900895292F30E0322F22274F
:1025500090E08C55914D280F391F81E020323105D4
:1025600008F080E008950F931F93CF93DF938C01C1
:10257000EB018A819B810E94A4128823A9F08981A2
:1025800081FF0DC080FD0BC06A816C55C8010E949F
:10259000A51181E0DF91CF911F910F9108958CE9F2
:1025A00093E00E940B14F5CF80E0F4CF6DE973E067
:1025B0008CE594E00E94872784E690E00E9428043E
:1025C0006AE08CE594E00E94AB2784E690E00E94EC
:1025D000280480E008950F931F93CF93DF93EC01BD
:1025E0008B0180EB93E00E943616998388831B83CE
:1025F0000A83CE010E943011CC5BDF4F8883DF91CC
:10260000CF911F910F910895BF92CF92DF92EF92D9
:10261000FF920F931F93CF93DF93EC018B0143E85D
:1026200053E08FEB93E00E94D019811186C047E000
:1026300050E06BE773E0C8010E946930892B09F014
:102640007CC0095F1F4F67E773E0C8010E946030DC
:10265000892B09F05FC08CE594E00E949325F12C52
:10266000E12C8A30910511F0019621F58A819B8138
:10267000E816F90608F04EC0888199818E0D9F1DDD
:102680000E942E114AE050E0682F8CE594E00E94F1
:10269000212884E690E00E94280460E28CE594E022
:1026A0000E94AB2784E690E00E9428048FEFE81A8E
:1026B000F80ADCCF8CE594E00E9493258A309105DE
:1026C00011F1019601F18A819B81E816F906D8F48F
:1026D00041E070E060E08CE594E00E949628B62E20
:1026E00067018FEFC81AD80A88819981E80EF91E10
:1026F000C7010E949F30B81621F06B2DC7010E94C0
:10270000A7307601D7CFCE010E943011FE01EC5BDD
:10271000FF4F80836FE673E0C8010E946030892B11
:1027200051F441E070E060E08CE594E00E9496286E
:10273000CE010E94A51181E001C080E0DF91CF9120
:102740001F910F91FF90EF90DF90CF90BF90089571
:10275000EF92FF920F931F93CF93DF9300D000D09F
:102760001F92CDB7DEB78C01F62EE72E6091C30421
:102770008FEF898382E88A83FB827C836D832FEFCE
:1027800032E84F2D572F85EB91E00E94E307C801F7
:102790004096F801E817F90741F02081211111C096
:1027A000218121110EC0F082E1820F900F900F90D5
:1027B0000F900F90DF91CF911F910F91FF90EF90AD
:1027C00008953296E7CFCF93DF9300D000D01F92C9
:1027D000CDB7DEB7AB019C01205F3F4FFC012E1748
:1027E0003F0751F08081841305C08181851302C0A9
:1027F000108211823296F3CF6091C3042FEF31E83B
:1028000085EB91E00F900F900F900F900F90DF915C
:10281000CF910C94E307CF92DF92EF92FF920F9348
:102820001F93CF93DF9300D000D01F92CDB7DEB7B8
:102830007C0120E1E20EF11C8C01DD24DA9481E8B8
:10284000C82EE016F106D1F0F80140815181411106
:1028500002C0552381F06091C304D982CA824B83A0
:102860005C836D832FEF31E885EB91E00E94E307F5
:10287000F801108211820E5F1F4FE3CF0F900F906F
:102880000F900F900F90DF91CF911F910F91FF90BC
:10289000EF90DF90CF9008950F931F93CF93DF9326
:1028A00000D000D01F92CDB7DEB78B016091C3047A
:1028B0002FEF32E8A80185EB91E00E94E3076091D9
:1028C000C3042FEF31E8A80185EB91E00F900F9042
:1028D0000F900F900F90DF91CF911F910F910C945B
:1028E000E3070F931F93CF93DF938C01005F1F4F7C
:1028F000EC010C171D0771F068817981898198813D
:10290000911102C0882321F085EB91E00E94CD0651
:102910002296EFCF80E0DF91CF911F910F91089524
:10292000FF920F931F93CF93DF93EC018B01FB0179
:10293000F0800E949F30F81621F06F2DCE010E948A
:10294000A730F801F1802196CE010E949F30F81641
:1029500021F06F2DCE010E94A730C801DF91CF91E9
:102960001F910F91FF900895CF92DF92EF92FF9207
:102970000F931F93CF93DF937C0162E070E080EBB5
:1029800093E00E943616EC01F701918380838C015D
:102990006C01F2E0CF0ED11C0C151D0540F4C801EE
:1029A0000E949F308F3F41F40F5F1F4FF5CF66E0CD
:1029B00071E0CE010E949014F701C081D181CE0157
:1029C0000E949F3080930601CE0101960E949F30A5
:1029D0008093070180E0DF91CF911F910F91FF90CD
:1029E000EF90DF90CF9008956FED73E08CE594E069
:1029F0000E94872784E690E00E9428046AE08CE524
:102A000094E00E94AB2784E690E00E94280480E0D6
:102A100008950F931F93CF93DF93EC018B0145EC47
:102A200053E08FEB93E00E94D019811144C06BEA10
:102A300073E0C8010E946030892BE9F58CE594E0D1
:102A40000E9493258A309105C9F00196B9F041E0C2
:102A500070E060E08CE594E00E94962860930601A7
:102A60007093070166E071E0888199810E9490145B
:102A700081E0DF91CF911F910F910895609107013F
:102A800070E0762F662780910601680F711D4AE07D
:102A900050E08CE594E00E94282884E690E00E94B3
:102AA000280460E28CE594E00E94AB2784E690E085
:102AB0000E942804D7CF80E0DCCFCF93DF93DC01E6
:102AC000EB019A818C91981305C02B8111968C9102
:102AD000281749F09E3721F080E0DF91CF910895CB
:102AE0008B81813DC9F7898181FFF6CF80FDF4CFCD
:102AF00087FDF2CF83E191E00E94CB1D882361F333
:102B000061E083E191E00E942F1E1A821B8281E026
:102B1000E4CF84E690E00C9428044AE050E0682F6B
:102B20008CE594E00E9421280E94891560E28CE5E2
:102B300094E00E94AB270C948915FF920F931F938A
:102B4000CF93DF93EC01F62E08811981C8010E9412
:102B50009F30F81621F06F2DC8010E94A730CE01DA
:102B6000DF91CF911F910F91FF900895F89481E02C
:102B70008093E00080E28093D800E9ECF0E01082DE
:102B80008FE19EE40197F1F700C000001DBA10929A
:102B900068001CBC10BE1FBA10927A0010926E0022
:102BA00010926F0010927100109272001082ECEB84
:102BB000F0E0108214B817B81AB81DB810BA108215
:102BC00015B818B81BB81EB811BA0C94003F089578
:102BD000AF92BF92CF92DF92EF92FF920F931F932B
:102BE000CF93DF9300D0CDB7DEB78C016C0184E0CA
:102BF000C80ED11C5601F12CE12CC7010E949F3058
:102C0000F50181935F01FFEFEF1AFF0A84E0E816F8
:102C1000F10499F7F80185818F3FD1F48481982FD1
:102C20009F779F3711F487FD148281E0F801858337
:102C300010E000E01A830983F60161916F01CE0173
:102C400001960E949D150F5F1F4F0430110591F7EB
:102C500080E00F900F90DF91CF911F910F91FF9027
:102C6000EF90DF90CF90BF90AF9008950F931F9398
:102C7000CF93DF9300D0CDB7DEB77A836983FC01B1
:102C8000238110E000E021110FC000811181CB01F0
:102C9000800F911F9183808342E0BE016F5F7F4F61
:102CA00088EB93E00E942518C8010F900F90DF91E8
:102CB000CF911F910F910895CF92DF92EF92FF92E3
:102CC0000F931F93CF93DF9300D0CDB7DEB77C0176
:102CD0006C0184E0C80ED11C10E000E01A83098367
:102CE000F60161916F01CE0101960E949D150F5F63
:102CF0001F4F0430110591F781E0F70182830F9097
:102D00000F90DF91CF911F910F91FF90EF90DF9087
:102D1000CF9008951F93CF93DF93EC01162F8091EE
:102D20000001681748F4862F0E9442098C81807840
:102D3000912F9F77892B8C831E3720F08C81807890
:102D40008E678C83CE010E945C168C818F77DF9119
:102D5000CF911F910895FC01948160FB97F99483B2
:102D6000892F8F778F3719F490789E679483CF01DE
:102D70000C945C16CF93DF93EC0181E08B8360E1D0
:102D800088EB93E00E940C188D81813021F01A822B
:102D9000DF91CF9108952E813F818091B80390916A
:102DA000B9032F3F320769F49F838E83CE010E94BF
:102DB0005C168C818F778E3758F7DF91CF910C940A
:102DC00042092817390721F7F4CFFC01238121118B
:102DD00002C00E94BA1680E0089584E090E09093CB
:102DE000B1038093B00308958CE594E00E9493258D
:102DF0009C0181E02A30310529F02F3F3F4F11F02F
:102E000080E0089508950F931F93CF93DF9300D030
:102E1000CDB7DEB78B0146E154E08FEB93E00E9423
:102E2000D019811135C066E074E0C8010E9460309D
:102E3000892BF1F40E94F41610E000E0811149C0E2
:102E40000E94F41681113DC041E070E060E08CE525
:102E500094E00E9496281A830983CE0101960E946D
:102E60009D150F5F1F4F011584E0180749F729C012
:102E70006AEF73E0C8010E946030892B59F06DEE53
:102E800073E0C8010E94603010E000E0892B69F116
:102E900080E018C08091B0039091B10360E074E0CD
:102EA000681B790B4AE050E08CE594E00E942828EA
:102EB0000E94891560E28CE594E00E94AB270E9495
:102EC000891581E00F900F90DF91CF911F910F91A5
:102ED0000895C8010E949F300E948D150F5F1F4FFB
:102EE000011584E01807A9F7ECCF1A8309836FEF67
:102EF000CE0101960E949D150F5F1F4F011584E0C2
:102F0000180799F70E94B615DCCFCF93DF93EB013A
:102F10004BE654E08FEB93E00E94D01981117AC008
:102F200049E050E061E674E0CE010E946930892BEF
:102F300009F070C0299664E574E0CE010E9460300B
:102F4000892B81F40E94F416811160C041E070E089
:102F500060E08CE594E00E94962880EB93E00E946C
:102F60008A1640C06DE474E0CE010E946030892B67
:102F7000E9F165E474E0CE010E946030892B71F1C3
:102F800061E474E0CE010E946030892B09F042C0F8
:102F90008091B303D0E0C0E0882321F0C091B60354
:102FA000D091B7036091B8037091B9034AE050E043
:102FB0008CE594E00E9428280E9489156FE374E054
:102FC0008CE594E00E9487270E9489154AE050E032
:102FD000BE018CE594E00E94282815C08091B503BD
:102FE0000E948D1581E0DF91CF9108956091B20329
:102FF0008FEB93E00E94071A0E94891560E28CE52E
:1030000094E00E94AB270E948915ECCF8091B40315
:103010008F77E6CF80E0E7CFFC01208131812170FE
:10302000332781E0861770F440815181569547958A
:1030300051834083220F331F41705527242B352B9A
:103040008F5FF0CF318320830895DC01FB01415075
:1030500000F181912D913C91119768E070E051E071
:10306000982F952399F4932F991F9927991F220F31
:10307000331F992319F095E029273058550F6150D7
:10308000710971F711963C932E93E1CF932F909590
:10309000EBCF089584E690E00C9428041F93CF931F
:1030A000DF939091BC03891730F080E090E0DF91CE
:1030B000CF911F910895C62FD0E094E5899FC00D50
:1030C000D11D1124CC0FDD1F6091BD037091BE0393
:1030D000C60FD71FCE010E949F30182FCE01019638
:1030E0000E949F30912FE3CF9091BB03891710F47A
:1030F0000C94FB08891B0C944E1880EB93E00E9403
:10310000E815809100018093BB0380E0089560E0A2
:1031100075E08CE594E00E9487270E944A186AE0D7
:103120008CE594E00E94AB270E944A1880E0089545
:103130008093BC0398EA899FB001112480EB93E04F
:103140000E9436169093BE038093BD03089580932A
:1031500000019091B4032EE438E197FD07C09091EF
:10316000BB03980F9093000124E738E130930301EB
:10317000209302010C949818FF920F931F93CF9302
:10318000DF9300D0CDB7DEB7F62E672F8C01000F8E
:10319000111F8091BD039091BE03800F911F9A83F0
:1031A0008983CE0101960E949D158091BD03909167
:1031B000BE030196800F911F9A8389836F2DCE01E4
:1031C00001960E949D150F900F90DF91CF911F9156
:1031D0000F91FF900895FF920F931F93CF93DF936A
:1031E000F82E8B01C0E0CF15F9F0D0E06D2F8C2FB9
:1031F000F8010995692F70E0762F6627680F711D19
:103200004AE050E08CE594E00E9428280E944A1889
:1032100060E28CE594E00E94AB270E944A18DF5FD1
:10322000D43521F7CF5FDFCFDF91CF911F910F9181
:10323000FF9008958CE594E00E9493259C0181E025
:103240002A30310529F02F3F3F4F11F080E00895DB
:103250000895FF920F931F93CF93DF931F92CDB7E3
:10326000DEB78B0141ED54E08FEB93E00E94D01963
:1032700081118EC047E050E069EC74E0C8010E9403
:103280006930892B09F084C0095F1F4F6EEB74E031
:10329000C8010E946030892BE1F50E941A19882329
:1032A000B1F06091B40367FB662760F94AE050E033
:1032B0008CE594E00E9421280E944A1860E28CE587
:1032C00094E00E94AB270E944A1881E062C041E06E
:1032D00070E060E08CE594E00E949628162F6983E8
:1032E00080EB93E00E94AB169091BC039093000199
:1032F000112339F08EE498E1909303018093020149
:10330000E4CF8091BB03890F8093000184E798E1AB
:10331000F3CF66EB74E0C8010E946030892B39F46A
:103320006BEF78E08091BB030E94EB18CECF6FEA81
:1033300074E0C8010E946030892B51F50E941A196F
:1033400010E000E094E5F92E882329F06EE478E19E
:103350008091BC03E9CF0E941A198111B6CF8091E8
:10336000BC038F9DC00111240817190708F0ADCFC9
:1033700041E070E060E08CE594E00E949628272F01
:103380003327722FC8010E94BC180F5F1F4FE3CF75
:1033900080E00F90DF91CF911F910F91FF900895E2
:1033A000CF93DF93CB01EA0167E475E00E946030C0
:1033B000892B49F4BE018CE594E00E94B62781E098
:1033C000DF91CF91089580E0FBCFCF93DF93EB01A6
:1033D0004DE255E00E94D019811117C060E275E0FE
:1033E000CE010E946030892B31F40E94B61581E035
:1033F000DF91CF91089568E175E0CE010E946030C1
:10340000892B19F40E949404F2CF80E0F1CF61116E
:1034100006C06DE075E08CE594E00C94872763E1CD
:1034200075E0F9CF1092DF030895CF93DF93EC019D
:103430008CE594E00E94A9258CE594E00E94AC25DF
:10344000892B09F45BC08CE594E00E94BC25E8A1BF
:1034500091E09E0F98A3EC0FFD2FF11D8083FE01DC
:10346000E90FF11D31978081803271F0903260F464
:103470008CE594E00E94AC25892B31F08CE594E03A
:103480000E9493250A97F9F68881811107C018A236
:1034900080E2FE0111928A95E9F730C0E8A1EC0FB5
:1034A000FD2FF11D319780818032F9F4E8A1E150C0
:1034B000FF0BEC0FFD1F8081803209F41082CE01DA
:1034C0000E9405058CE594E00E94AC25892B31F023
:1034D0008CE594E00E94BC258A30A1F76CE475E08D
:1034E0008CE594E00E94B627D2CF8CE594E00E9450
:1034F00093250A97D9F288A18032C0F680E0DF9147
:10350000CF91089560E575E08CE594E00E948727EF
:1035100084E690E00E9428046AE08CE594E00E9432
:10352000AB2784E690E00E94280480E00895CF93C2
:10353000DF9300D000D000D0CDB7DEB789E895E0AA
:103540000E94FA2EEDE9F5E0108A8685978524859C
:10355000358519823B832A839D838C831E82028456
:10356000F385E02D0190F081E02D46E050E0BE01B2
:103570006F5F7F4F87EA95E0099580E026960FB64A
:10358000F894DEBF0FBECDBFDF91CF910895FC014F
:10359000703579F4862F8076803429F49085862FD3
:1035A0008F7B892B8087862F807729F48781682BF2
:1035B000678380E008958031E1F780E1689FB00182
:1035C0001124F4CFCF93DF93EC0189E895E00E94BA
:1035D000BD2E688589E895E00E94C32E89E895E0B4
:1035E000DF91CF910C94D52EFB01928196FB22277F
:1035F00020F980E090FD82E0822B20E091FD24E024
:10360000822B20E092FD28E0822B93FD04C090E005
:10361000892B0C943F1C90E1FBCFFB0123812035CB
:1036200059F4DC0117961C9217972281322F3076BD
:10363000303421F418961C9280E0089525FFFCCFC9
:10364000218121FFF9CF20FDF7CF0E94F41AF4CF9A
:103650002091B6013091B701FC013183208396811E
:10366000892F8F7019F41092EB0308958091100147
:10367000819592FF80E093FF03C020911001820F9B
:1036800060911001619590FF60E091FF03C09091FF
:103690001001690F0E94E11C89E895E00C94D52E79
:1036A0000F932091B6013091B701FC01358324833B
:1036B000868190E024E0959587952A95E1F700971B
:1036C000F1F000910A01019582FF00E083FF03C041
:1036D00020910A01020F20910A0180FF20E081FF62
:1036E00003C080910A01281B40E060E089E895E072
:1036F0000E94B52E89E895E00F910C94D52E0F917C
:103700000895CF93DF93EC018091B6019091B701BA
:103710002A813B81AC01421B530B9A0140910B0162
:1037200050910C012417350780F09B838A832091E8
:10373000EB0330910D014FEF50E0431B510924176B
:1037400015061CF4230F2093EB0328813981821B7B
:10375000930B20910E0130910F018217930718F0FF
:10376000CE010E94281B8091B6019091B7012C8157
:103770003D81821B930B2091080130910901821732
:10378000930718F0CE010E94501B80E0DF91CF918B
:1037900008950F931F93CF93DF93FB01238120356F
:1037A000C9F48B01EC0182818076803419F4CE015A
:1037B0000E94E21A8F818E831F82F80182818077B6
:1037C00079F48091B6019091B7019B838A83CE01F1
:1037D0000E94281B80E0DF91CF911F910F910895E7
:1037E0008031C1F7CE010E94501BF4CFCF93DF93FD
:1037F00000D000D000D0CDB7DEB736952795820F28
:10380000931F56954795640F751FEDE9F5E0958771
:10381000848777876687208929839B838A837D8332
:103820006C831E820284F385E02D0190F081E02DEF
:1038300046E050E0BE016F5F7F4F87EA95E0099553
:1038400026960FB6F894DEBF0FBECDBFDF91CF91A5
:1038500008951092EE031092ED031092F00310926F
:10386000EF038FEF9FE79093F4038093F30390931C
:10387000F2038093F10381E08093EC0308950F93AA
:103880001F93CF93C82F8091EC03811102C00E9437
:10389000291CC0FF06C01092EC03CF911F910F911D
:1038A0000895E09112010E2F10E08091F3039091A2
:1038B000F403B8010E94D52F9B017093F403609329
:1038C000F3038091F1039091F203B8010E94D52F88
:1038D000AB017093F2036093F1036C2F6470E0917D
:1038E000EF03F091F0038091ED039091EE037C2FB4
:1038F0007670763091F4820F931F9093EE0380934D
:10390000ED03BA016E0F7F1F7093F0036093EF0316
:10391000CF911F910F910C94F61B662349F1D801AA
:103920001197A49FB001A59F700DB49F700D112435
:10393000E60FF71FF093F003E093EF03C4FF1DC001
:1039400001501109029FB001039F700D129F700D6D
:103950001124860F971F9093EE038093ED036091DF
:10396000EF037091F0038091ED039091EE03D0CFBF
:10397000C1FDE4CFE40FF51FDDCFC3FDF0CF820F13
:10398000931FE9CF482F50E087FD0AC0889FC001F0
:103990001124880F892F881F990B91958F5F0895A7
:1039A00020E031E0241B350B229FC001239F900DA6
:1039B000900D1124880F892F881F990B9195809560
:1039C0000895EF92FF920F931F93CF93DF93082FE9
:1039D000162FC0911101D0E0F12CE12C8823D1F0F9
:1039E0008091EB030E94C21C2091EA03382F03034D
:1039F000C0011124820F911D27FD9A957E01C817E1
:103A0000D90744F0EE24FF24EC1AFD0AE816F90663
:103A10000CF47C01112309F449C08091EB030E944E
:103A2000C21C2091E903382F1303C0011124820F17
:103A3000911D27FD9A95C817D9073CF0D195C195DE
:103A4000D109C817D9070CF4EC011092EC03AE01B0
:103A5000D7FF02C0415F5F4F94E0559547959A9517
:103A6000E1F7B701F7FE02C0615F7F4F84E0759513
:103A700067958A95E1F700E020E089E895E00E94EB
:103A8000B52E20E130E0C701B9010E94E92F8093F3
:103A9000EA03CE01B9010E94E92F8093E903DF9187
:103AA000CF911F910F91FF90EF900895D0E0C0E06B
:103AB000CCCFFC018281DB019C91891730F5A0817C
:103AC000B181A80FB11D2C9130E0938102C03595D2
:103AD00027959A95E2F724834481442391F0242F7B
:103AE00030E0938140FF07C0880F880F880F890F4F
:103AF000858381E008953595279524839F5F93837F
:103B0000EBCF8F5F82831382D5CF80E00895262F7D
:103B1000269526952695820F911DFC01808190E0C7
:103B2000677002C0959587956A95E2F78170089550
:103B3000E62FE695E695E695E80FF92FF11D6770FB
:103B400081E090E0A0E0B0E004C0880F991FAA1FB8
:103B5000BB1F6A95D2F72081822B80830895E62FC0
:103B6000E695E695E695E80FF92FF11D862F87700B
:103B700041E050E060E070E004C0440F551F661F54
:103B8000771F8A95D2F74095509560957095808102
:103B9000482340830895EF92FF920F931F93CF9392
:103BA000DF93CDB7DEB72C970FB6F894DEBF0FBE0C
:103BB000CDBF8C010A9698878F8319861A86FF24B9
:103BC000FA94FC869A8389838BE0E82EEB821C8230
:103BD000FE82BE016D5F7F4FCE0107960E94591D88
:103BE000811113C00B5E1F4F18870F8319861A8629
:103BF000FC861A830983EB821C82FE82BE016D5F04
:103C00007F4FCE0107960E94591D2C960FB6F8944F
:103C1000DEBF0FBECDBFDF91CF911F910F91FF90FF
:103C2000EF900895272F207C69F4605E683098F447
:103C3000FC018681978102C0969587956A95E2F787
:103C400081700895743439F426ED260F2A3218F461
:103C50006252603168F381E008950C94121EAF92B5
:103C6000BF92DF92EF92FF920F931F93CF93DF9358
:103C7000CDB7DEB761970FB6F894DEBF0FBECDBFEC
:103C80008C010A967C01662381F1580195E1A90E09
:103C9000B11CB886AF8219861A868FEF8C87BA82DC
:103CA000A9829BE09B831C828E83BE016D5F7F4F48
:103CB000CE0107960E94591D8823B9F0DC846D2D32
:103CC000C5010E94AF1D6D2DC7010E94AF1D6091FF
:103CD000C3042D2D31E84FEF5FEF85EB91E00E949B
:103CE000E3078A858F5F8A87E0CFF886EF8219869F
:103CF0001A868FEF8C87FA82E9829BE09B831C8275
:103D00008E830B5E1F4FBE016D5F7F4FCE01079606
:103D10000E94591D882309F1DC846D2DC8010E9481
:103D2000871D6D2D8823A9F0C8010E94AF1D6D2D40
:103D3000C7010E94AF1D6091C3042D2D31E84FEFE4
:103D40005FEF85EB91E00E94E3078A858F5F8A87AA
:103D5000DACFC7010E94AF1DF8CF61960FB6F89475
:103D6000DEBF0FBECDBFDF91CF911F910F91FF90AE
:103D7000EF90DF90BF90AF9008956AE575E08CE515
:103D800094E00E94872784E690E00E9428046AE07D
:103D90008CE594E00E94AB2784E690E00E94280422
:103DA00080E008954F925F926F927F928F929F92E0
:103DB000AF92BF92CF92DF92EF92FF920F931F9339
:103DC000CF93DF93CDB7DEB761970FB6F894DEBF20
:103DD0000FBECDBF8C01FC0160807180C090B60128
:103DE000D090B70180A191A1C81AD90A828093808E
:103DF0007801FAE0EF0EF11CF886EF8219861A8638
:103E00008FEF8C87FA82E9829BE09B831C828E83F2
:103E1000512C580185E1A80EB11CBE016D5F7F4F8A
:103E2000CE0107960E94591D482E882349F15C84D3
:103E3000652DC5010E94871D8823D1F0C614D704C3
:103E400090F0652DC5010E94AF1D652DC7010E9430
:103E5000AF1D6091C304252D31E84FEF5FEF85EB77
:103E600091E00E94E3078A858F5F8A87542CD5CF23
:103E7000C814D904C0F3652DC7010E94AF1DF3CF4C
:103E8000511007C08091B6019091B701F80191A33C
:103E900080A380E061960FB6F894DEBF0FBECDBF61
:103EA000DF91CF911F910F91FF90EF90DF90CF9016
:103EB000BF90AF909F908F907F906F905F904F904A
:103EC00008950C94D21E872F90E0982F8827860F94
:103ED000911D2FEF280F283018F4815290E008959B
:103EE0008F5D94E40895AF92BF92CF92DF92EF92EC
:103EF000FF920F931F93CF93DF93FB01B180B7FC29
:103F00005BC0EB018C016C01FAE0CF0ED11C688123
:103F1000C6010E94871DA82E780185E1E80EF11CDC
:103F20006881C7010E94871DB1FE90C0B0FC8EC0A1
:103F3000A11051C0811185C08A819B81292F30E059
:103F4000322F2227482F50E04150504C240F351F6C
:103F50002031310598F46A817B81C8010E94631F7A
:103F60009B838A836881C6010E94981D8091B60157
:103F70009091B701F80191A380A31BC0F80120859F
:103F8000222339F0292F207C21F420E2280F283029
:103F900048F3F8012185222331F0943421F426EDF1
:103FA000280F2A32F8F2292F207C41F4805E8830D5
:103FB00050F48881F80182A380E038C0943419F469
:103FC0008A528A32B0F3F80180A191A12081318117
:103FD000821B930BD0CF882361F36881C6010E94B6
:103FE000AF1D9881F80182A1981729F06881C70157
:103FF0000E94AF1DDECF6A817B81C8010E942D1E09
:104000008823A1F3F8018481958197FF02C0808104
:1040100091812091B6013091B701F80140A151A1E1
:10402000241B350B2817390708F782E0DF91CF9161
:104030001F910F91FF90EF90DF90CF90BF90AF90C6
:1040400008956881C6010E94AF1DD0CFA11003C0A2
:10405000882309F4B1CF6881C7010E94981DE5CF7C
:1040600062E675E08CE594E00E94872784E690E0A4
:104070000E9428046AE08CE594E00E94AB2784E665
:1040800090E00E94280480E00895FC01872F90E0D2
:10409000982F8827680F792F711D613180EC780780
:1040A000E0F0623188EC780750F46151704C66A7FB
:1040B00017A611AA80EE870F80AB81E008956331C7
:1040C00080ED780750F46251784C66A717A68AE213
:1040D000870F80AB84E481ABF0CF80E008958F92AE
:1040E0009F92AF92BF92CF92DF92EF92FF920F9387
:1040F0001F93CF93DF9300D000D0CDB7DEB78C01F4
:10410000F62E23E5261708F469C0E62FF0E0EE0F3F
:10411000FF1FEC53FB4FD080E1808FEFD8120FC010
:10412000E8120DC0AF2DB0E0A554BE4FE0910201E2
:10413000F09103016F2D8C910995D82EE92E6D2DEC
:104140007E2DC8010E944520B82E811135C0EF2D6B
:10415000F0E0E554FE4F8080C12CAA24AA94912C53
:10416000F8018281C81608F042C0F4E0CF9EC00179
:104170001124F80160817181680F791FAA8244E0DF
:1041800050E0CE0101960E94573089819A813B818F
:104190002C81F9122AC0482F082E000C550B481507
:1041A000590511F08F3F09F5F801D6A6E7A6C90118
:1041B00090AB21ABBB24B3948B2D0F900F900F903D
:1041C0000F90DF91CF911F910F91FF90EF90DF90B3
:1041D000CF90BF90AF909F908F90089510926C05F4
:1041E00010926D05ECE6F5E096CFC394B9CFD6A654
:1041F000E7A68FEF80AB81ABDFCFCF93DF93FC01DE
:10420000EB019A01261B370BA4E6B0E00E94253093
:1042100026A130E050E040E00E94FD2F8091B601E1
:104220009091B701BC016C1B7D0B81E06217730795
:1042300008F080E0DF91CF910895292F207C39F498
:1042400090E2980F81E0983048F080E007C0943405
:10425000E1F796ED980F81E09A32B8F70895CF9381
:10426000DF93EC018881681780F5882371F1815014
:104270008883E62FF0E0DF011196AC0FBD1FEE0F33
:10428000FF1F7196EC0FFD1F962F981780F4119663
:104290002C9111972D9318962C91189717962C9373
:1042A000179722813381219331939F5FEECF2FEFB8
:1042B00030E001C0220F6A95EAF789A1922F90950C
:1042C000982386958223892B89A3DF91CF91089526
:1042D000CF93DF9300D000D01F92CDB7DEB7FC01A3
:1042E000348584A1982F917080FD28C082E02481BC
:1042F00039838A836B837C832D8391110AC0872F36
:1043000090E0982F8827680F792F711D6430710510
:10431000F0F460E0CF0103960E942F2129813A81B9
:104320004B815C816D8185EB91E00F900F900F9038
:104330000F900F90DF91CF910C94970881E0D7CF29
:104340006D32710530F36933710518F703C06832B7
:104350007105B0F78489958994A783A7DACFCF93A5
:10436000DF93FC017381DC011D9681E090E060E049
:104370008717F0F452A94D9124A130E0082E02C015
:10438000359527950A94E2F720FD0DC0541721F0CA
:1043900080E0DF91CF9108952489358934AB23AB38
:1043A000682F0196E5CF5413FCCF8FEF82ABF0CF8F
:1043B0008091B6019091B70123A934A9821B930B78
:1043C00025A92817190609F068F48FEF82AB662338
:1043D000F9F2EF012396CE010E942F2160E0CE0179
:1043E0000E942F2181E0D5CF7F928F929F92AF9232
:1043F000BF92CF92DF92EF92FF920F931F93CF93D2
:10440000DF93EC019B81911110C0F12C8F2DDF9176
:10441000CF911F910F91FF90EF90DF90CF90BF90C1
:10442000AF909F908F907F9008959C848CA180FF87
:1044300013C0983041F460E070E0CE010E94682122
:10444000FF24F394E3CF8AA99812F5CFCE010E94FE
:10445000AF218111DACFEFCF692DCE010E946F20FD
:10446000882309F470C0FDA0FF2009F46CC00EA5DC
:104470001FA5C8010E941D21882E8091B601909130
:10448000B7012BA53CA5821B930B2AA5281719065B
:1044900009F010F57B80A090B601B090B7016E01D5
:1044A00001E010E0E12C202F071508F065C08CA179
:1044B00090E0002E02C0959587950A94E2F780FD62
:1044C00012C0811040C0EE2009F454C07FEFC71A1B
:1044D000D70A0F5F1F4FE7CF8110DCCFB801CE01A5
:1044E0000E946821D7CFF6019585FE013D9681E0B7
:1044F00099122DC0EE2019F08EA1811110C08820D4
:1045000059F068A979A99AAA8C899D899CAB8BAB33
:10451000CE010E9468217ACF6EA57FA5F4CFF80165
:10452000EE0FFF1FEC0FFD1F44895589EE2DF0E0C3
:10453000EE0FFF1FEC0FFD1F64897589CE010E94ED
:10454000FD208111C3CF6EA57FA577CF8F5F821726
:1045500008F0BCCF31913913F9CF4C895D89B50191
:10456000641B750B39A53617170609F078F768A98B
:1045700079A9CECFE02EAACF88E0781246CFE3CF3C
:104580000F931F93CF93DF93EC01FB0124818DA543
:10459000922F981B19162CF08B8181111CC080E082
:1045A00025C02DA780818435D0F7818187FDF7CF85
:1045B0008B018DA181111FC062817381CE010E9488
:1045C0004520882361F38EA59FA5D80113969C935F
:1045D0008E931297E4CF022E000C330B8C81281B94
:1045E000310987FD339537FDDACF82E0DF91CF9136
:1045F0001F910F9108952B81822F90E03481FE014D
:10460000E80FF91F3483DB013C913487880F991F31
:10461000FE01E80FF91F8091B6019091B701958BCB
:10462000848B11964C913CA181E090E0A0E0B0E039
:10463000022E04C0880F991FAA1FBB1F0A94D2F72D
:1046400040FF0CC041FD0AC0832B8CA32F5F2B833E
:10465000CE010E94F4218111FBCFC7CF8095832327
:10466000F4CF0F931F93CF93DF93EC012091B6010A
:104670003091B7018AA590E04BA55CA5B901641BF8
:10468000750B6817790738F0A90141505109481B8B
:10469000590B5CA74BA78B818823D9F08C899D8906
:1046A000281B390B8FA198A52817390768F00EA58C
:1046B0001FA5C8010E941D21B801811102C068A96F
:1046C00079A9CE010E946821CE010E94F4218111B6
:1046D000FBCF80E0DF91CF911F910F910895CF9391
:1046E000DF93C5EFD3E0198218821A821B8288E01B
:1046F000EBE4F1E0A1E0B4E001900D928A95E1F7DE
:1047000081E08DA380E58EA38AEF90E098A78FA328
:1047100082E389A78BE48AA780E091E09CA78BA71E
:104720008FEF8DA78EA78FA788AB89AB8AAB88EC5C
:104730008DABDF91CF910895FC018FEF81831282C1
:10474000409153015091540160915501709156016F
:104750004783508761877287848B809140048111E1
:104760002CC081EE809348041092490486E2809325
:104770004A0488E080934B0410924D0410924C043C
:1047800095EE90934E0410924F0497E2909350044C
:1047900080935104109253041092520410925404C6
:1047A0001092550410925604109257041092590416
:1047B0001092580481E08093400488E494E0909340
:1047C0005B0480935A04089569E675E08CE594E0F3
:1047D0000E94872784E690E00E9428046AE08CE526
:1047E00094E00E94AB2784E690E00E94280480E0D9
:1047F000089580E026E0E0915A04F0915B04829FE6
:10480000E00DF11D1124908191110FC03181311102
:104810000CC03281311109C03381311106C044818D
:104820005581452B11F48FEF0895961303C09181A4
:10483000971711F08F5FDFCF08950F931F93CF93DA
:10484000DF93CDB7DEB72A970FB6F894DEBF0FBE61
:10485000CDBF8C01FC01838980FD48C082E0F80156
:10486000278193812E838F838FEF888789879A870B
:10487000662321F1948997FD21C09081923079F4CB
:104880006091C304298391E09A838B838C836D8329
:1048900031E04FEF5FEF85EB91E00E94E307F80115
:1048A0008489E0915A04F0915B0496E08902E00D5E
:1048B000F11D11248281938199878887F801828173
:1048C0008823E1F0815082833396D8011B9690E0D3
:1048D000981770F4218121932481238312962D91BE
:1048E0003C9113972D933D939F5FF2CF81E0B7CF1B
:1048F000F801838990E095958795838B2E813F8180
:10490000488559856A8585EB91E02A960FB6F8941B
:10491000DEBF0FBECDBFDF91CF911F910F910C94E1
:104920009708CF93DF93EC018A81882329F060E018
:10493000CE010E941D24F8CFDF91CF910895FC0194
:104940008281882311F120913601309137018489C9
:10495000A0915A04B0915B0496E08902A00DB11DAC
:10496000112414968D919C91009709F09C018091DF
:10497000B6019091B70143855485841B950B82172E
:10498000930718F0CF010E94912480E00895CF93FF
:10499000DF93FC01EB012081822F90E03C81DF015D
:1049A000A80FB91F11963C931197388115963C9327
:1049B000880F991FDF01A80FB91F8091B601909150
:1049C000B7011A969C938E9319979981818941E03A
:1049D00050E060E070E0022E04C0440F551F661FD7
:1049E000771F0A94D2F790FF09C091FD07C0482BAA
:1049F000418B2F5F2083DF91CF910895409548230D
:104A0000F7CF0F931F93CF93DF93EC01FB018481CA
:104A10009981282F291B12164CF09A8191111CC0E4
:104A200080E0DF91CF911F910F91089589832081BC
:104A30002435B0F7818187FDF3CF382F327081FFA5
:104A40001FC080FD1DC09281983591F49381913DE6
:104A5000B9F4188281E0E5CF082E000C990B2B8168
:104A6000821B910927FD939597FDDACF82E0D9CF7C
:104A7000993531F49381913D19F481E08883D1CF48
:104A80009881913069F28F019A81992371F080FFAA
:104A900009C0311107C08F81821323C061E0CE01AC
:104AA0000E941D24CE010E949124F801818181FF82
:104AB000B7CF80FDB5CF62817381CE010E94F9230B
:104AC0008C8B87FDADCF8881823069F4F80120811D
:104AD000318142815381648185EB91E00E94E3073B
:104AE00002C09430F9F2B801CE0102960E94C724A8
:104AF000BDCF8BE294E00C949C23CF93DF931F9265
:104B0000CDB7DEB76983DC01ED91FC910280F381C2
:104B1000E02D41E050E0BE016F5F7F4F09950F909F
:104B2000DF91CF910895CF93DF93EC018C859D8524
:104B300097FF05C082E00E94E9299D878C878C85BC
:104B40009D85DF91CF91089583E00E94002A90E037
:104B5000089583E00C946F2CFC018485958597FD66
:104B600006C082E00E94992990E00196089582E0B3
:104B70000E94992990E00895FC018485958597FD10
:104B800005C02FEF3FEF35872487089582E00C940E
:104B9000E929CF93DF93EC0180914301882331F021
:104BA00083E00E941A2A1816190634F081E090E07A
:104BB0009B838A8380E090E0DF91CF910895EEEFB0
:104BC000FFE72591349181E02B3F3C4D09F080E0D7
:104BD0000895FC0190819E5F908342E450E064E779
:104BE00075E080E80C94CB2AFC0181819081913A98
:104BF00061F4813209F083C047E050E06CE371E07A
:104C000080E00E94CB2A81E00895913209F077C0BC
:104C1000833269F482819381B0E0A0E0809338010F
:104C200090933901A0933A01B0933B01ECCF8032CD
:104C300039F467E070E08CE391E00E94F12AE3CF61
:104C4000823209F78281809343010E94DF25E0E0F0
:104C5000F8E0882311F0EEEFFAE080913C019091AA
:104C60003D01A0913E01B0913F01803B9440A105E0
:104C7000B105D9F48091430180FD17C0EE3F8AE071
:104C8000F80771F587E797E791838083809160004B
:104C90008093AC0488E19BE00FB6F894A8958093CC
:104CA00060000FBE90936000AECF80819181873706
:104CB000974709F0A8CFA8958091600088618093FC
:104CC00060008091AC0480936000EE3F8AE0F807BA
:104CD00089F08091FE0A9091FF0A9183808393CF9F
:104CE000808191818737980769F29093FF0A8093BA
:104CF000FE0AC8CF1092FF0A1092FE0A84CF80E00D
:104D000008952FEF3FEFFC01358724870895ECE5E8
:104D1000F4E01382128288EE93E0A0E0B0E0848396
:104D20009583A683B7838BE791E0918380838FEF90
:104D30009FEF958784870895EF92FF920F931F93BB
:104D4000CF93DF937B01FC01C281D38110E000E0AF
:104D5000209791F0E881F9810280F381E02DB7017D
:104D6000CE01099597FD06C0080F191F0884D98543
:104D7000C02DEECF0FEF1FEFC801DF91CF911F9134
:104D80000F91FF90EF9008950F931F93CF93DF93B0
:104D90008B01FC01C281D381209771F0E881F981F8
:104DA0000480F581E02DB801CE010995009731F41A
:104DB0000884D985C02DF0CF90E080E0DF91CF91BD
:104DC0001F910F9108950F931F93CF93DF938B0142
:104DD000FC01C281D381209771F0E881F9810680BE
:104DE000F781E02DB801CE010995080F111D088447
:104DF000D985C02DF0CFF8011082DF91CF911F919E
:104E00000F9108950F931F93CF93DF938B01FC01B4
:104E1000C281D381209771F0E881F9810190F081FE
:104E2000E02DB801CE010995811105C00884D9850E
:104E3000C02DF0CF80E0DF91CF911F910F910895A9
:104E4000CF93DF93FC01DB01218114968C911497A1
:104E5000820F9927991F08978CF5C281D3812097DB
:104E600031F573836283908112969C931297139607
:104E70002C93139715968C911597890F808380E05A
:104E800014969C9114978917E8F41696CD91DC91AD
:104E90001797C80FD11D9881C181D0E0CC5BDE4F40
:104EA000988391819F5F91838F5FEACFEC01888522
:104EB00099850097D9F7B987A887D5CF80E0DF918A
:104EC000CF91089581E0FBCF8091AD0481110DC099
:104ED00082E08093B50484E08093B6041092B80415
:104EE0001092B70481E08093AD0485EB94E00895BF
:104EF000FB0101900020E9F73197AF01461B570BEA
:104F0000DC01ED91FC910280F381E02D0994EF9298
:104F1000FF920F931F93CF93DF938C017B01D0E01F
:104F2000C0E0F701EC0FFD1F6491662361F0D8012A
:104F3000ED91FC910190F081E02DC8010995892B3C
:104F400011F02196EECFCE01DF91CF911F910F91FD
:104F5000FF90EF900895DC01ED91FC910190F081BC
:104F6000E02D099469E871E00C9478270F931F9362
:104F7000CF93DF93EC010E9487278C01CE010E9422
:104F8000B227800F911FDF91CF911F910F9108954C
:104F90008F929F92AF92BF92EF92FF920F931F93C7
:104FA000CF93DF93CDB7DEB7A1970FB6F894DEBFEE
:104FB0000FBECDBF7C01FA01CB0119A2223008F44B
:104FC0002AE08E010F5D1F4F822E912CB12CA12C57
:104FD000BF01A50194010E94FD2FF901CA016A30A9
:104FE0000CF5605DD8016E938D01232B242B252BAE
:104FF00079F790E080E0109721F0BD01C7010E9491
:105000007827A1960FB6F894DEBF0FBECDBFDF9113
:10501000CF911F910F91FF90EF90BF90AF909F9015
:105020008F900895695CDECF2115310541F4DC01D4
:10503000ED91FC910190F081E02D642F09940C9486
:10504000C8279A01462F50E070E060E00C941428C5
:105050009A01AB0170E060E00C9414280F931F9349
:10506000CF93DF93EC010E94BE03688779878A871C
:105070009B87E881F9810484F585E02DCE010995AF
:1050800097FF15C00E94BE03088519852A853B85B8
:10509000601B710B820B930B0C811D812E813F8154
:1050A000601771078207930720F38FEF9FEFDF915F
:1050B000CF911F910F910895FF920F931F93CF935C
:1050C000DF93EC018B01F42ECE010E942E2897FD78
:1050D0001DC08D329105D1F09C01205331092A3039
:1050E0003105A0F0FF2019F08E32910579F00130E2
:1050F000110551F00230110589F48D30910571F0E0
:105100005CF40997029750F08FEF9FEFDF91CF91FA
:105110001F910F91FF9008958097B1F7E881F98171
:105120000284F385E02DCE010995CECFBF92CF92B8
:10513000DF92EF92FF920F931F93CF93DF938C0137
:10514000C42F40E00E945C28FC01C12CD12C7601C8
:1051500097FD3EC0B12C0C2E000CDD0BCE17DF07E7
:10516000D9F0ED32F10509F43FC0CF01C0970A979D
:1051700098F4AAE0B0E0A70196010E9434306F01D4
:10518000FF0FEE08FF08C60ED71EE81EF91E80E3CB
:10519000C81AD108E108F108D801ED91FC91028408
:1051A000F385E02DC8010995C8010E942E28FC0155
:1051B000C0970A9798F2CE17DF0781F2BB2041F023
:1051C000F094E094D094C094C11CD11CE11CF11C5B
:1051D000C701B601DF91CF911F910F91FF90EF9022
:1051E000DF90CF90BF900895BB24B394D5CF40916A
:1051F000BC045091BD042091BA043091BB04421705
:105200005307B4F49091E8009570E1F39091E800B1
:1052100092FD19C08093F1008091BC049091BD046F
:1052200001968F739927892B19F48EEF8093E800EC
:105230008091BC049091BD0401969093BD0480932D
:10524000BC0481E0089580E00895EF92FF920F93EF
:105250001F93CF93DF93F82E192FE62E042F81E0B2
:10526000860F880F0E94F72883E00E94F728CF2D31
:10527000D12FEC0EFD2EF11CCE15DF05B9F007FF86
:1052800013C0FE0184910E94F728182F80E00E942D
:10529000F728812321968111EFCFDF91CF911F91C4
:1052A0000F91FF90EF9008958881EDCF81E0F5CFC9
:1052B0008091D70081608093D70080EA8093D800E6
:1052C00089B5806189BD89B5826089BD09B400FE58
:1052D000FDCF61E070E080E090E00E94EF038091FC
:1052E000D8008F7C80618093D8008091E000807F1F
:1052F0008093E0000895CF93DF931F92CDB7DEB780
:105300001982CE0101960E94E9250E946427BE0100
:105310006F5F7F4F0E949C2689810F90DF91CF9114
:1053200008952FB7FC012083F89467706093E9001B
:105330000895CF93DF931F92CDB7DEB7682FCE01CC
:1053400001960E9491298091F20099819FBF0F9050
:10535000DF91CF910895EF92FF920F931F93CF9318
:10536000DF931F92CDB7DEB79091C004992371F1FE
:1053700057FD2CC08A017B01682FCE0101960E9447
:1053800091298091F20090E0081719070CF4C801E8
:10539000282FF70144E6215030F04093C1043091AA
:1053A000F1003193F8CF009739F02091F2002111EC
:1053B00003C02BE62093E80029812FBF0F90DF91D7
:1053C000CF911F910F91FF90EF9008958FEF9FEF76
:1053D000F5CFCF93DF931F92CDB7DEB741E050E01A
:1053E000BE016F5F7F4F0E94AB29019731F4898125
:1053F00090E00F90DF91CF9108958FEF9FEFF9CF5D
:10540000CF93DF931F92CDB7DEB7682FCE01019601
:105410000E9491299091E800892F807295FF04C025
:105420009091F20080E4891B99819FBF0F90DF91DA
:10543000CF9108955F926F927F928F929F92AF92D9
:10544000BF92CF92DF92EF92FF920F931F93CF9371
:10545000DF931F92CDB7DEB7982E6B01B42E052FC8
:105460008091C004811113C08FEF9FEF0F90DF91E7
:10547000CF911F910F91FF90EF90DF90CF90BF9051
:10548000AF909F908F907F906F905F9008958091E4
:10549000BE0480FF05C08091E00082608093E00040
:1054A000EB2CF02EA12C8AEF882E892D8072682E8D
:1054B000892D8074582E9AE3792EE114F10419F4A1
:1054C000AA2009F457C0892D0E94002A182F8111A3
:1054D0000AC08A94882041F261E070E080E090E0A8
:1054E0000E94EF03EACF8E151F0411F00CF01E2D61
:1054F000692DCE0101960E9491298091E80085FDD9
:1055000003C089818FBFD9CF812F90E0E81AF90AB3
:10551000662029F01150A0F01092F100FBCFF601A7
:1055200097FC0AC0115050F021912093F100FACF5E
:1055300024912093F10031961150D0F7C80ED91E56
:10554000AA2021F07092E800A12CDBCF8091E80026
:1055500085FD08C07092E800AA24A394E114F10428
:1055600081F2F2CFE114F10461F6552051F270920C
:10557000E800C7CF84E68093C2048B2D902F76CFAE
:105580001092E9001092BD041092BC049093BB04E9
:105590008093BA040895DF92EF92FF920F931F93C6
:1055A000CF93DF93D82E8A01EB017B01E40EF51E29
:1055B000CE15DF0559F0D7FE12C0FE0184910E947E
:1055C000F72821968111F4CF0FEF1FEFC801DF916B
:1055D000CF911F910F91FF90EF90DF9008958881F8
:1055E000EECFCF93DF93EC019B01B4E6ABEF211537
:1055F0003105F1F0A9012134310514F040E450E007
:105600008091E80082FFFCCF942FFB01E21BF30B9B
:10561000EC0FFD1F915028F08091F10080833196AE
:10562000F9CFB093C104A093E800241B350BDFCF62
:10563000CB01DF91CF9108951F920F920FB60F9279
:105640001124CF92DF92FF920F931F932F933F93DA
:105650004F935F936F937F938F939F93AF93BF937A
:10566000EF93FF93CF93DF93CDB7DEB76C97DEBF99
:10567000CDBF1092E9008091E80083FF2FC089E040
:10568000FE017596FE2E0F2F815029F09091F100AA
:1056900090833196F9CF84E68093C10482EF8093A2
:1056A000E8008D8987FF38C09091E80090FFFCCF1B
:1056B000982F907609F000C19E894F89588D2F89C7
:1056C000188D911130C0803859F58091BF048093B6
:1056D000F1001092F1008EEF8093E8006C960FB607
:1056E000F894DEBF0FBECDBFDF91CF91FF91EF9158
:1056F000BF91AF919F918F917F916F915F914F91EA
:105700003F912F911F910F91FF90DF90CF900F90BD
:105710000FBE0F901F9018959EEF9093E800C8CF92
:105720001092F100D6CF913059F48111D4CF41308D
:10573000510589F68091BF048D7F8093BF04CBCF44
:10574000933049F48111C7CF4130510521F6809142
:10575000BF048260F2CF953041F48091E80080FF71
:10576000FCCF20682093E300B6CF963009F076C0D6
:10577000CB8CDC8C123039F590E080E00E94C02A9E
:105780000E947B291F8299E099831A8391E09E836E
:1057900090EA98879AEF99872091BC043091BD04D4
:1057A000275F3F4F3C832B838D83C6010E94C02A15
:1057B00049E050E0BE016F5F7F4F80E00E94CB2A3E
:1057C0000E947B2988CFC6010E94C02A0E946427BC
:1057D0006F2D702F0E94C426009731F00CF07BCF04
:1057E00081E28093EB007ACF113061F11330C1F781
:1057F0008F89882381F1823049F440E86AE083EDA3
:1058000095E00E942529882359F365CF813029F43A
:1058100040E86AE088EC95E0F4CF833009F70E9415
:1058200064278E010F5F1F4FB8010E94E326F80125
:1058300001900020E9F73197BF01601B710B40E038
:10584000C801DFCF66EB75E0FB01449150E080E8D2
:105850000E94CB2A40CF6EED75E0F6CF973009F469
:10586000BFCF983021F481E08093F10034CF99309C
:1058700009F031CF837009F0B3CFE5E4F1E081E0C6
:1058800031E096E32191222371F08093E900309377
:10589000EB00DF0111972C912093EC009093ED0029
:1058A0008F5F873079F78EE78093EA001092EA00E5
:1058B0008F898093C0040FCF8B8D9C8D0E94C02A4E
:1058C000898D811105C08F2D902F0E94F4259BCFCB
:1058D0000E9464276F2D702F0E94022794CF80931F
:1058E000E9008091F200882319F08AE38093E800B0
:1058F00008951F920F920FB60F9211242F933F938A
:105900004F935F936F937F938F939F93AF93BF93C7
:10591000CF93EF93FF93C091E1008091E100837FEB
:105920008093E100C3FF0FC01092E90081E08093F3
:10593000EB001092EC0082E38093ED001092C00423
:1059400088E08093F000C2FF15C083E00E946F2CB6
:105950008091C204882329F08091C20481508093F1
:10596000C2048091C104882329F08091C104815030
:105970008093C104C4FF23C08091E2008E7E8160C9
:105980008093E2008091E1008F7E8093E10080911E
:10599000BE048E7E80618093BE04FF91EF91CF9113
:1059A000BF91AF919F918F917F916F915F914F9137
:1059B0003F912F910F900FBE0F901F901895C0FF31
:1059C000ECCF8091E2008E7E80618093E200809136
:1059D000E1008E7E8093E1008091BE048E7E816026
:1059E000DACF1092C0041092BF041092BE040E943D
:1059F0005829E1EEF0E080818E7E80838DE08093F7
:105A0000E200559A209A08958091E0008D7F80935E
:105A1000E0008091E00081FD11C08091BE0480FF14
:105A20000DC08091BF0481FF09C00E945829809158
:105A3000E00082608093E00081E0089580E00895B6
:105A4000089510926C0510926D050895CF93DF9321
:105A5000CDB7DEB769970FB6F894DEBF0FBECDBFE6
:105A6000FC01DB018C918F5F8C939E012D5F3F4F7A
:105A70008DE0D9011D928A95E9F729E0298384E018
:105A80008A8391E09D8383E08E832A8721E22B879E
:105A90009C879D879F8722E2288B27E02B8B25E020
:105AA0002C8B8E8B20E430E0388F2F8B998F828166
:105AB0008B8395858685998B8A8B838180688D8B76
:105AC00049E150E0BE016F5F7F4F80E00E94CB2A2A
:105AD00069960FB6F894DEBF0FBECDBFDF91CF91B0
:105AE0000895EF92FF920F931F93CF93DF93FB01E3
:105AF00020812138A1F52381223289F5DC0112961B
:105B00004C91248135814217130649F5EC0181E05F
:105B10000E94D42F0B851C85F12CE12C0115110559
:105B200089F0F801448155816281738180E80E9487
:105B3000CB2A8F3F980761F0E80EF91ED8010D912E
:105B40001C91ECCF81E08F8780E00E94D42FC701A9
:105B5000DF91CF911F910F91FF90EF90089590E00A
:105B600080E0F6CFCF93DF93EC01DB012A8114961E
:105B70008D919C9115972817190659F411968C91BF
:105B800011979C91913A39F4982F9D7F81E0913043
:105B900051F080E008C09132E1F78B3039F4129671
:105BA0008C918F8781E0DF91CF9108958A3021F425
:105BB00013968C91888BF6CF893059F716968D9174
:105BC0009C918230910539F462E070E0CE014196FB
:105BD0000E94F12ADECF0197E1F661E070E0CE018C
:105BE00042960E94F12A198AD4CFFC01A385B4857C
:105BF000109771F47487638785859685DB01149609
:105C00002D913C91820F931F968785870895DC0123
:105C10008D919C9111970097D1F76D937C93ECCF68
:105C2000AF92BF92CF92DF92EF92FF920F931F93AA
:105C3000CF93DF931F92CDB7DEB77C0169836A01F2
:105C4000590141E050E0BE016F5F7F4FFC0183814D
:105C50000E941A2A8C0197FD0BC0F7018381A501D0
:105C6000B60180640E941A2A080F191F97FD8C0143
:105C7000C8010F90DF91CF911F910F91FF90EF908E
:105C8000DF90CF90BF90AF900895CF92DF92EF92C8
:105C9000FF921F93CF93DF93162F7A0169010E9421
:105CA000102EEC01E091E002F091E102309729F032
:105CB0009C01A601B701812F0995CE01DF91CF91FB
:105CC0001F91FF90EF90DF90CF900895CF93DF93D7
:105CD000EC0181E08C838D839E01265F3F4F3F83E3
:105CE0002E831986188620E931E0398328831C86A3
:105CF0001B861E861D868F87888B198A1A8A81ECDF
:105D00008A870E946427BE01DF91CF910C942027DF
:105D100080916E05811107C086E795E00E94662E8E
:105D200081E080936E0586E795E00895FC01158279
:105D300080918F05811113C01092980510929705DC
:105D400082EE95E090939A05809399058AE390E01E
:105D500090939C0580939B0581E080938F050E9422
:105D6000882E67E975E00C94F52D0F93FC01618393
:105D70004283238304830F91089525E0FC0111924F
:105D80002A95E9F70895FC019081692B60830895B5
:105D9000CF93DF93EC010E94882E25E030E0AE0126
:105DA00061E0DF91CF910C94452ECF93DF93EC010E
:105DB00098818D8198130CC08981811109C08A81D5
:105DC000811106C08B81811103C08C81882329F049
:105DD000CE010E94C82E88818D83DF91CF910895D6
:105DE000CF93DF93EC010E94BD2ECE01DF91CF91C6
:105DF0000C94D52E0C94F02E89E895E00C94962EF8
:105E0000CF93DF93CDB7DEB769970FB6F894DEBFB7
:105E10000FBECDBFFC01DB019C919F5F9C939E0157
:105E20002D5F3F4F81E1D9011D928A95E9F729E065
:105E3000298384E08A8391E09D8383E08E832A878F
:105E400021E22B879C879D879F8722E2288B25E371
:105E5000298B27E02B8B25E02C8B8E8B20E430E0E8
:105E6000388F2F8B998F82818B83838180688D8B74
:105E700049E150E0BE016F5F7F4F80E00E94CB2A76
:105E800069960FB6F894DEBF0FBECDBFDF91CF91FC
:105E900008950F931F93CF93DF93EB018A01FC01C9
:105EA000838180640E941A2AE091E002F091E1026D
:105EB000309749F09C01A801BE0187E0DF91CF91A6
:105EC0001F910F910994DF91CF911F910F91089528
:105ED0000A970C94492FDC01FB0112962C91129722
:105EE000848195812817190641F491818081813A36
:105EF00031F49D7F81E0913009F080E00895813296
:105F0000E1F79B3029F4828152968C9381E00895C9
:105F10009A3099F7828153968C93F8CFFB012081B8
:105F20002138B1F42381223299F4DC0112964C918C
:105F30001297248135814217130651F421E05296BD
:105F40002C9345E350E06CE176E080E80C94CB2A9A
:105F500090E080E00895CF93DF93EC0181E08C83A3
:105F60008D839E012F5E3F4F3F832E8319861886B7
:105F70001D861C861F861E86188A2CE931E039830F
:105F800028832AEA31E03B872A878A8B8B8B81EC36
:105F9000898B0E946427BE01DF91CF910C9420274A
:105FA0008DE995E00C94AB2F0895AA1BBB1B51E122
:105FB00007C0AA1FBB1FA617B70710F0A61BB70B79
:105FC000881F991F5A95A9F780959095BC01CD011E
:105FD000089597FB072E16F4009407D077FD09D09B
:105FE0000E94D52F07FC05D03EF4909581959F4FD8
:105FF0000895709561957F4F0895A1E21A2EAA1B0E
:10600000BB1BFD010DC0AA1FBB1FEE1FFF1FA21768
:10601000B307E407F50720F0A21BB30BE40BF50B65
:10602000661F771F881F991F1A9469F760957095EE
:10603000809590959B01AC01BD01CF010895EE0FB5
:10604000FF1F0590F491E02D0994A29FB001B39F2A
:10605000C001A39F700D811D1124911DB29F700D71
:10606000811D1124911D08950E942530A59F900D3A
:10607000B49F900DA49F800D911D112408950024BC
:10608000A7FD00942A0F301D401D501D601D701D7E
:10609000801D901D08950024A7FD00942A17300547
:1060A0004005500560057005800590050895FB01C9
:1060B000DC0102C005900D9241505040D8F7089580
:1060C000FB01DC018D91059080190110D9F3990B2A
:1060D0000895FB01DC014150504030F08D91059056
:1060E000801919F40020B9F7881B990B0895FB015A
:1060F000DC0104C08D910190801921F44150504081
:10610000C8F7881B990B0895FB01DC0102C00190C0
:106110000D9241505040D8F708956817790768F4F8
:10612000FB01DC01E40FF51FA40FB51F02C00290B4
:106130000E9241505040D8F708950C948430F9994C
:10614000FECF92BD81BDF89A992780B50895262F7C
:10615000F999FECF1FBA92BD81BD20BD0FB6F8944C
:0E616000FA9AF99A0FBE01960895F894FFCFAF
:10616E0003FFFB080101290032000140000101007C
:10617E00017F02C409FA00FFFFFFFF0000000000CC
:10618E000000000000000000000000000000000001
:10619E000000000000FFC800FFFFFFFF00E100004D
:1061AE000000000000C18081000000FFFFFFFFFF24
:1061BE00FFFFFFFFFFFFFF4572676F446F782D45AE
:1061CE005A00B50130313233929366000000001D43
:1061DE000EB50D000EAE0D000000007D25C925A4E4
:1061EE0025A925AC25BC2593250D0A00000000002D
:1061FE00B22D262D712D8A04000000006B2F002F6A
:0C620E008E2FAE0D492FF6FF0000682F08
:00000001FF
